:020000040000fa
:080000000002040000000000f2
:020000040000fa
:04000800f0050000ff
:020000040000fa
:04000c00f0050000fb
:020000040000fa
:04001000f0050000f7
:020000040000fa
:04001400f0050000f3
:020000040000fa
:04001800f0050000ef
:020000040000fa
:04001c00f0050000eb
:020000040000fa
:04002000f0050000e7
:020000040000fa
:04002400f0050000e3
:020000040000fa
:04002800f0050000df
:020000040000fa
:04002c00f0050000db
:020000040000fa
:04003000f0050000d7
:020000040000fa
:04003400cc030000f9
:020000040000fa
:04003800f0050000cf
:020000040000fa
:04003c00f0050000cb
:020000040000fa
:04004000f0050000c7
:020000040000fa
:04004400f0050000c3
:020000040000fa
:04004800320300007f
:020000040000fa
:04004c00f0050000bb
:020000040000fa
:04005000f0050000b7
:020000040000fa
:04005400d0050000d3
:020000040000fa
:04005800b4050000eb
:020000040000fa
:04005c00f0050000ab
:020000040000fa
:04006000f0050000a7
:020000040000fa
:04006400f0050000a3
:020000040000fa
:04006800bc020000d6
:020000040000fa
:04006c00f00500009b
:020000040000fa
:04007000f005000097
:020000040000fa
:04007400f005000093
:020000040000fa
:04007800f00500008f
:020000040000fa
:04007c00f00500008b
:020000040000fa
:04008000f005000087
:020000040000fa
:04008400f005000083
:020000040000fa
:04008800f00500007f
:020000040000fa
:04008c00f00500007b
:020000040000fa
:04009000f005000077
:020000040000fa
:04009400f005000073
:020000040000fa
:04009800f00500006f
:020000040000fa
:04009c00f00500006b
:020000040000fa
:0400a0007a040000de
:020000040000fa
:0400a40076040000de
:020000040000fa
:0400a800f00500005f
:020000040000fa
:0400ac00f00500005b
:020000040000fa
:0400b000f005000057
:020000040000fa
:0400b400f005000053
:020000040000fa
:0400b800f00500004f
:020000040000fa
:0400bc00f00500004b
:020000040000fa
:0400c000f005000047
:020000040000fa
:0400c400f005000043
:020000040000fa
:0400c800f00500003f
:020000040000fa
:0400cc00f00500003b
:020000040000fa
:0400d000f005000037
:020000040000fa
:0400d400f005000033
:020000040000fa
:0400d800f00500002f
:020000040000fa
:0400dc00f00500002b
:020000040000fa
:0400e000f005000027
:020000040000fa
:0400e400f005000023
:020000040000fa
:0400e800f00500001f
:020000040000fa
:0400ec00f00500001b
:020000040000fa
:0400f000f005000017
:020000040000fa
:0400f400f005000013
:020000040000fa
:0400f800f00500000f
:020000040000fa
:0400fc00f00500000b
:020000040000fa
:04010000f005000006
:020000040000fa
:04010400f005000002
:020000040000fa
:04010800f0050000fe
:020000040000fa
:04010c00f0050000fa
:020000040000fa
:04011000f0050000f6
:020000040000fa
:04011400f0050000f2
:020000040000fa
:04011800f0050000ee
:020000040000fa
:04011c00f0050000ea
:020000040000fa
:04012000f0050000e6
:020000040000fa
:04012400f0050000e2
:020000040000fa
:04012800f0050000de
:020000040000fa
:04012c00f0050000da
:020000040000fa
:04013000f0050000d6
:020000040000fa
:04013400f0050000d2
:020000040000fa
:04013800f0050000ce
:020000040000fa
:04013c00f0050000ca
:020000040000fa
:04014000f0050000c6
:020000040000fa
:04014400f0050000c2
:020000040000fa
:04020800f0050000fd
:020000040000fa
:04020c00f0050000f9
:020000040000fa
:04021000f0050000f5
:020000040000fa
:04021400f0050000f1
:020000040000fa
:04021800f0050000ed
:020000040000fa
:04021c00f0050000e9
:020000040000fa
:04022000f0050000e5
:020000040000fa
:04022400f0050000e1
:020000040000fa
:04022800f0050000dd
:020000040000fa
:04022c00f0050000d9
:020000040000fa
:04023000f0050000d5
:020000040000fa
:04023400cc030000f7
:020000040000fa
:04023800f0050000cd
:020000040000fa
:04023c00f0050000c9
:020000040000fa
:04024000f0050000c5
:020000040000fa
:04024400f0050000c1
:020000040000fa
:04024800320300007d
:020000040000fa
:04024c00f0050000b9
:020000040000fa
:04025000f0050000b5
:020000040000fa
:04025400d0050000d1
:020000040000fa
:04025800b4050000e9
:020000040000fa
:04025c00f0050000a9
:020000040000fa
:04026000f0050000a5
:020000040000fa
:04026400f0050000a1
:020000040000fa
:04026800bc020000d4
:020000040000fa
:04026c00f005000099
:020000040000fa
:04027000f005000095
:020000040000fa
:04027400f005000091
:020000040000fa
:04027800f00500008d
:020000040000fa
:04027c00f005000089
:020000040000fa
:04028000f005000085
:020000040000fa
:04028400f005000081
:020000040000fa
:04028800f00500007d
:020000040000fa
:04028c00f005000079
:020000040000fa
:04029000f005000075
:020000040000fa
:04029400f005000071
:020000040000fa
:04029800f00500006d
:020000040000fa
:04029c00f005000069
:020000040000fa
:0402a0007a040000dc
:020000040000fa
:0402a40076040000dc
:020000040000fa
:0402a800f00500005d
:020000040000fa
:0402ac00f005000059
:020000040000fa
:0402b000f005000055
:020000040000fa
:0402b400f005000051
:020000040000fa
:0402b800f00500004d
:020000040000fa
:0402bc00f005000049
:020000040000fa
:0402c000f005000045
:020000040000fa
:0402c400f005000041
:020000040000fa
:0402c800f00500003d
:020000040000fa
:0402cc00f005000039
:020000040000fa
:0402d000f005000035
:020000040000fa
:0402d400f005000031
:020000040000fa
:0402d800f00500002d
:020000040000fa
:0402dc00f005000029
:020000040000fa
:0402e000f005000025
:020000040000fa
:0402e400f005000021
:020000040000fa
:0402e800f00500001d
:020000040000fa
:0402ec00f005000019
:020000040000fa
:0402f000f005000015
:020000040000fa
:0402f400f005000011
:020000040000fa
:0402f800f00500000d
:020000040000fa
:0402fc00f005000009
:020000040000fa
:04030000f005000004
:020000040000fa
:04030400f005000000
:020000040000fa
:04030800f0050000fc
:020000040000fa
:04030c00f0050000f8
:020000040000fa
:04031000f0050000f4
:020000040000fa
:04031400f0050000f0
:020000040000fa
:04031800f0050000ec
:020000040000fa
:04031c00f0050000e8
:020000040000fa
:04032000f0050000e4
:020000040000fa
:04032400f0050000e0
:020000040000fa
:04032800f0050000dc
:020000040000fa
:04032c00f0050000d8
:020000040000fa
:04033000f0050000d4
:020000040000fa
:04033400f0050000d0
:020000040000fa
:04033800f0050000cc
:020000040000fa
:04033c00f0050000c8
:020000040000fa
:04034000f0050000c4
:020000040000fa
:04034400f0050000c0
:020000040000fa
:10040000cfe521000eff27000e018800000000004c
:10041000000020000000e000020032000001200087
:10042000200288000e000700e02b220001002000bf
:10043000810f70000100320014000700000020004e
:100440000000e00002003200000002000000000096
:100450002c260200000000000040da000000fe0030
:100460004440a900400520000000e00003003200e5
:1004700000002000a00188004440a8000000060001
:100480008a1f78008b1f7800000006009101880009
:10049000800478000000eb001a003700e28444007a
:1004a00032a0b4009905ba00e284440032a0b4003e
:1004b0009906ba00e284440032a0b4000006eb00c2
:1004c000476fde00fd07b200636ce10003003a00f5
:1004d000ebff07000000eb000a003700606ce10052
:1004e00004003a00005deb008b05e900fdff3e00d3
:1004f000040037006168e100010032000086eb0073
:100500000b00070019c7ba001905ba000e04e00075
:1005100003003a000a00e000e0ff3a000000060095
:10052000fe07b2009e0188008a047800f5ff3700bc
:10053000395dba008b05e9000c003200295dba0074
:100540008b05e900080032000c00e00003003a00cf
:10055000e284440032a0b400f5ff370019ddba0090
:100560008b05e900faff3a008904e800e1844400c1
:1005700032a0b400000006003600f800809fbe00e4
:10058000829fbe00849fbe00869fbe0008a2ab0073
:1005900011003a000010800042e8b7000842ab00aa
:1005a0000a00320044c8bf004b0c07000000fb00eb
:1005b000101088000782a8000802ab00feff3a0076
:1005c00030c0b30043e8b7001f00370010c0b300cd
:1005d00043e8b7001c00370043c8bf00e14f50009c
:1005e00007003a000010800044e8b7000782a80026
:1005f00020c0b30043e8b7004568ef0012003700a1
:10060000e24f500005003a000110800044c8bf00ce
:10061000ce0c07000782a8000b003700e34f500004
:1006200009003a0044c8bf004548b4002a0c07003e
:100630000000fb00101088000782a8000802ab0031
:10064000feff3a004568ec008600a9004f03be009b
:100650004f02be004f01be004f00be003600f90041
:10066000004006003600f800809fbe00829fbe005a
:10067000849fbe00869fbe00889fbe008a9fbe00ea
:100680001800fa0008ff2f00a01680000004640084
:10069000f00f440029003a0070408000e10f500044
:1006a00010003c0005c8bf00e14f500008003a00b0
:1006b0000568ef00bc0807000000eb000000000028
:1006c0000000e800f40f5000fcff3a009109070019
:1006d0008800780000852000520d07000e28ec00ed
:1006e0001400370080408000e10f500011003a00f4
:1006f000fa8457000004eb004a0e20004b932000c0
:1007000008004400f88057000080400088407800ce
:10071000950807000ac0b90000804500d90078009c
:10072000400d07000804e800ec0f5400f4ff3a0005
:100730001028ef001628ef000d0037001008e20027
:1007400007003a001608ec00b0408800e60f5000a1
:1007500003003a00100020008040880005e8b70040
:100760000e28ef0088007800008520002d0d07007e
:100770008500a9000080fa004f05be004f04be00ae
:100780004f03be004f02be004f01be004f00be002f
:100790003600f900004006003600f800809fbe00d9
:1007a000829fbe00849fbe00869fbe00881f780087
:1007b0005816800023c8bf00e14f50000a003a00dd
:1007c0002008ec0000418800e1022000810f500069
:1007d00002003a002028ef002368ef00ca22ef0051
:1007e0008460a9003a00370024c8bf00e14f5000e0
:1007f0001f003a002468ef002248e2000e003a0091
:100800004dc8bf000080fb008711070010c0b30077
:1008100022e8b7005166210011088800612c2000f1
:100820006108880031162000110c8800010c880036
:1008300023e8b7000e0037004cc8bf000080fb0063
:10084000791107002268ef0000fa200010088800e4
:100850009005200060088800c0022000100c88006d
:10086000000c88001e68ef0010c0b30023e8b7003a
:10087000680cb2001ec8bf00e14f50000f003a00e4
:10088000004180008000400062602100e28078002a
:10089000088470000000e80000418800e1022000a8
:1008a000810f500008003a002028ef001e68ef007a
:1008b00010c0b30024e8b7000300370060602100d7
:1008c0002b1107001ee8b700581688008460a900a5
:1008d0004f0478004f03be004f02be004f01be0020
:1008e0004f00be003600f9000040060087e0a90076
:1008f000004006003600f800809fbe00829fbe00c8
:10090000849fbe00869fbe00881f78003200fa00d8
:1009100087c0a900b01180000000fb00cf80de007e
:100920001003b1000180b10052032000820f50007b
:10093000e08f58005b003e00006001005b00370064
:100940007d0037007e00370032003700330037006b
:1009500034003700350037003600370037003700e5
:10096000500037004f0037004e0037004d00370071
:100970004c0037004b0037004a0037003d0037007d
:100980003e0037003f00370040003700410037008d
:100990004200370043003700420037004100370073
:1009a000400037003f0037003e0037003d00370071
:1009b0003c0037003b0037003a0037003900370071
:1009c0003800370037003700360037003500370071
:1009d0003400370033003700320037003100370071
:1009e000300037002f0037002e0037002d00370071
:1009f0002c0037002b0037002a0037001100370089
:100a000012003700130037001400370015003700bc
:100a10001600370042002000250037005200200059
:100a20002300370062002000210037007200200000
:100a30001f003700820020001d00370092002000b8
:100a40001b003700a200200019003700b200200070
:100a500017003700c200200015003700d200200028
:100a600013003700e200200011003700f2002000e0
:100a70000f003700a20020000d003700b200200058
:100a80000b003700c200200009003700d200200010
:100a900007003700e200200005003700f2002000c8
:100aa000030037000081eb00010037001200200036
:100ab0002dc8bf008000fb0081804000e382200041
:100ac00082b178000040e8002de8b700e34f500005
:100ad0001d0034002d68ef0003007800100478003a
:100ae0004c44dd0090009000c808dd000104440083
:100af000b000900001044400200090004400dd009c
:100b00000004440008007800c40d0700881f780026
:100b100000432900801f7800a0fc2f000f00400038
:100b2000f0030700a0fc2f000f004000e40d0700b9
:100b3000e48757000400370022002000dcff370064
:100b400032002000daff37000080fa004f047800fe
:100b50004f03be004f02be004f01be004f00be005b
:100b60003600f90000400600809fbe008580a90085
:100b700038c8bf00eb4f500007003c00b141800077
:100b80008100e800b14188009100fb00211188003c
:100b90000040e80038e8b7004f00be000040060003
:100ba0003600f800809fbe00829fbe00849fbe007a
:100bb000869fbe008560a900311180008100fb0086
:100bc00020ac2100170c07004f03be004f02be00ef
:100bd0004f01be004f00be003600f9000040060085
:100be0000040da000000fe0000c0da00000006004d
:100bf0000a00fa00e20f500034003e00d0f28000fc
:100c0000e10f500003003200e20f500011003a00e3
:100c10000c003700032220000300e00001003a002e
:100c20000040da002002e200020035002822ef0036
:100c300021e2a8002342ab000d003a002342a800a5
:100c40000b003700032320000300e00001003a00fe
:100c50000040da003002e200020035003822ef00e6
:100c600031e2a8003342ab0001003a003342a80051
:100c7000820178000b0037003102fb00e10f5000c9
:100c800004003a002322ab00feff3a002411880042
:100c9000030037003322ab00feff3a00a4118800a6
:100ca0008301e9000300e000f3ff3a00e10f500088
:100cb00003003a002302ab00feff32000b003700b6
:100cc0003302ab00feff3200080037003300200083
:100cd000b3bf9f00c0bf9f00d1bf9f00e2bf9f0076
:100ce0006a805700c0ff07006fb9970002007800c4
:100cf0000080fa00000006006011b80066013700ad
:100d0000889fbe008a9fbe008c1f7800910107005b
:100d10009801330003866c006450e1002400320027
:100d20006420e100270032006150e100220032001f
:100d30006120e100210032008b854200eb07b10009
:100d40000134b800003ab8000804420089844a001f
:100d5000013ab8000030b8008880400009014a001c
:100d60000400330000004000818048000201490077
:100d70008b05e900c909dd00830170000100320024
:100d800013002000c814de004814dd004709de000f
:100d90001200b200c808de00088470008501070058
:100da00001f0a1000cf0a70001f0a0007a013700cb
:100db0006120e1007c0132000801be000200be009b
:100dc000f7ff37006150e100fcff3a007601370081
:100dd00003f0a200889fbe008a9fbe008c1f78008f
:100de0005c010700630133006450e1004f003200f2
:100df0006420e1005200320003826c0007003b00d7
:100e00000905d0000306d000820f54000c065d00d7
:100e100002003900020032008901780003067800e0
:100e20008582550004003d000003fd008103fd00a4
:100e30008502ea008b854200840f720002003b00ad
:100e400060001000e08018006011b8000005eb00a1
:100e50007a28e1000a00390006007800c75ddd004d
:100e6000f707b200878075002d003700828171007e
:100e70000a017800610560008180d1000080d30004
:100e80008502e900f9ff3b00060440008784480022
:100e900002003b0060041400e0841c000988a300e9
:100ea000070032008a817100828171006101640053
:100eb0008904d1000884d3008b05e80017003700af
:100ec0000978a30013003a000b00e000130034007f
:100ed0008b05e9000804440089844c000a4474002e
:100ee0000978a3000d003a000b00e0000700340071
:100ef0008b05e9000804440089844c0001003a0095
:100f00000b0020000978a300f7ff32000001eb007e
:100f100002003700828171000a0178002501070074
:100f20000cf0a70001f0a0001b0137006420e100d5
:100f300002003a00838f6c001b0133000801be00e1
:100f40000200be0014013700040020003f013700fa
:100f5000889fbe008a9fbe008c1f7800fd0007009e
:100f60001002200002003b0070428800010137009f
:100f70008a0062006408e10002003a0070428800c2
:100f8000090137006108e100fcff32000800be00e3
:100f9000030478000d00070001f0a10046010700de
:100fa00008f0a600040037000001be0091042400f0
:100fb000b0fd200086ff070009f0a70001f0a200a5
:100fc000f50037000081eb00a0013700889fbe00cc
:100fd0008a9fbe008c1f7800de000700e50033000a
:100fe00003866c006450e1002e0032006420e100b2
:100ff000330032006150e1002f0032006120e10037
:101000003100320085855500eb07b0000900200053
:1010100008042000050037000804440089844c00bf
:101020000a0031000603430087834b000001530090
:1010300081815b00f8ff33000203be000800a000be
:101040000804440089844c00f6ff3900c639dd00ed
:101050008301730001003200130020008904d100d5
:101060000884d3000998a300050032000800a700f7
:101070000300a0008904d1000884d3008b05e80098
:101080008904d1000884d3000001eb000281d20062
:10109000c800070001f0a1000cf0a70001f0a000bb
:1010a000bd0037006420e100bf0032000801be002f
:1010b0000200be00f7ff37006120e100ba003200f5
:1010c0006000b800f3ff37000000200001f827009f
:1010d000f0ff3700889fbe008a9fbe008c1f7800fb
:1010e0000004be00c20107000478a30026003a00f5
:1010f0006120e1002500320009f8a30025003a0034
:101100006420e10021003200f507b1000508a300ca
:101110000200320000004000818048006044b800b6
:1011200003102000020020000000400081804800e1
:101130000805440089854c000a0541008b8549005b
:101140000a0550008b855800030033000a00be00da
:1011500002047400838474008301d1000281d300ef
:10116000830f7100f0ff3a008904d1000884d30096
:101170006001490082017800c1adde00fb07b000cc
:101180008c000700840037000960a0000800be0042
:10119000810037001202200072428800f0ff2f0009
:1011a000f1ff27007c0037000001be00900107001e
:1011b0000470a70003f0a1006509b1001600320019
:1011c0000d0035006828e10006003500f0ff2f0013
:1011d000f1ff27000300e00013003b00010028009e
:1011e0000000050000004000818048008502e90001
:1011f000fcff3a0008003700f88f420002003c0074
:101200008000eb00000005008100d1000080d300c9
:101210008502e800fcff3a000300e00002003b000a
:1012200060001000e0801800000006000001be0011
:101230006f0107000470a70003f0a10003f8a300ea
:1012400013003a006509b1001000320009003500b2
:101250006928e100020035000100280000000500b7
:1012600000004000818048008502e900fcff3a0050
:1012700000000600f88f4200050035008100d10013
:101280000080d3008502e800fcff3a000000060061
:101290008000eb0000000500889fbe008a9fbe0012
:1012a0000082700004027100048271002600320086
:1012b0000004be000200be006011b8006b092000ef
:1012c000950220000182cf000a0039000541b100db
:1012d0000082cf00070039000541b1000982cf002c
:1012e000040039000541b1000882cf000100390037
:1012f0000541b10005425200120032000a003b00d5
:1013000082817100610164008100d1000080d300fe
:101310008984d3000884d3008b05e8000442e800e8
:10132000f7ff3a00070037000804440089844c00a6
:1013300000004800818048008b05e9000442e90074
:10134000f9ff3a001b0007004f05be004f04be0026
:10135000000006000004be00250107000003be00d7
:101360000405be000200be0021010700844f750085
:10137000000006000200be006450e10005003600d7
:101380006420e100020036000968a30001003a0071
:101390000800be000160a0004f0678004f05be00a7
:1013a0004f04be0000000600f0ff2f00f1ff2700f1
:1013b000f9ff370081002000618055000b003d00df
:1013c0000b00200061fe2f000100e1001d00340031
:1013d00082817100610164008904d1000884d30016
:1013e0000000e800faff3a0071002000610064008c
:1013f0000300700002006000090032006104440034
:10140000e0844c000988a500050032008b05e80047
:101410006808e10002003a008904d1000884d30082
:10142000f20f20000258e10005003d00c75ddd001d
:10143000f907b200898075000800780000000600f6
:101440000bf827008b00780000000500889fbe0085
:101450008a9fbe00841f7800beff07004f007800ff
:1014600011003300f0ff2f00838f6c0006003b005b
:10147000040565000a00a7000800370009f0a6006f
:101480001000200008003700820f5400838f5c009a
:10149000030039001000200001003e000000200081
:1014a00009f0a7000000ea004f05be004f04be008f
:1014b0000000e00000000600889fbe008a9fbe007a
:1014c0008c9fbe000004be00c90007000800be00db
:1014d000890678006420e100080039000400320029
:1014e0000160a00012022000724288005300370001
:1014f00091fc2300b0fd20004e0037000006eb00f9
:1015000009f0a10003f82300020020000800be003b
:10151000cc0007000600340001f823000000200082
:101520000801be00a9fe07000004be002c00200038
:101530000800be0093e82300320a2300c100070020
:10154000120034000801be00d1fd2300703d2b00c5
:1015500020fe07000005be00b3f32300f27a260048
:101560000800be00e6fd070003f82300020020008b
:1015700017fe07000801be0016fe07000a01be00a4
:1015800092fe07000004be000c06e8000800be0042
:1015900001f0a1000200200003982300a900070029
:1015a0000800be00160035000801be00d4fd07008b
:1015b0000005be0032cd2c0043fb230005fe0700d2
:1015c000809fbe001269280003d52b000a00be00d0
:1015d000cbfd0700620f210013ef2b00fdfd07007c
:1015e0000a01be00c6fd07004f01be0077fe0700de
:1015f0000801be00c2fd07000801be00f5fd07009e
:101600000c00e0000b0032000c10a70001f0a2005b
:10161000b2fd200093fc23006260e1000400320070
:1016200022a9200063f023000c10a70063f8230018
:10163000e8fd07000df0a70001f0a2004f06be0074
:101640004f05be004f04be0000000600889fbe008c
:101650008a9fbe008c9fbe00820578000004be00f9
:10166000630007000800be006420e10007003900a5
:1016700002003a00f1ff2700f0ff2f000160a000f8
:101680001202200072428800550037006120e100fc
:1016900003003a000b00a70001f8230050003700b8
:1016a00001f0a100020021009364240065000700fe
:1016b0000800be0004003500b2fd2000930c240099
:1016c000620007000004be000005eb000b00a6004e
:1016d0004f0dde0001f0a1000004be0032982f0083
:1016e00023ea230086fd07000001eb0003f023003e
:1016f0000b00a70003f82300b6fd0700aafe0700b1
:101700000000a7000a00a200520007000b00e00042
:10171000030032000200200003f02300acfd0700ac
:1017200001f0a2000006be00020020009304240085
:1017300073fd07000801be00a6fd0700809fbe00e4
:101740000c00be0022a22a00d3a723006cfd0700d4
:101750004f01be009ffd07000004be0001f0a10084
:101760000200200003982300360007000800be0096
:10177000190035000001be0061fd07000006be0033
:10178000b2c52900e36223005dfd070022222b0081
:10179000f3942b008ffd07000c01be0058fd0700dd
:1017a000e273280083c023008afd07000c01be00fd
:1017b00053fd070042aa2a00a3e22b0085fd070083
:1017c0000c01be004efd07000801be004cfd0700e5
:1017d0000801be007ffd07000a00a70001f0a2007b
:1017e0004f06be004f05be004f04be0000000600bd
:1017f000c70ade00f107b200f50fb20008003200a0
:10180000e1cf4200020032000170a0002400050078
:10181000810f70000100320004080500440005003b
:10182000810f700002003a00140005008502e900f3
:101830000000400081c04800fcff3b000170a00098
:10184000240005001400200000ff370004002000e1
:10185000030037004f89de00820178004f00370017
:10186000889fbe008a9fbe008c1f78004f26dd0037
:10187000b8fe0700bffe33006120e10043003200e4
:101880006250e10041003e003e0039006420e1006a
:101890003c003200058255000f003b000402e800c6
:1018a00038003a00800f5300818f5b003500340010
:1018b0000800be0003f0a10001f0a60003f0a000a4
:1018c0000cf0a70043fd0700b3fe370006034300fa
:1018d00087834b000c4646000005530081855b0062
:1018e000020033000a03be000c00a0000402e9005d
:1018f000f6ff3b00850578000602430087824b0017
:1019000004003a006000b80009f0a70001f0a00050
:10191000a1fe37000002520081825a000704e00055
:10192000040033000603430087834b008b05e90066
:10193000faff3700090578000604be000203be0066
:101940006011b8009bfe0700e00f5200e08f5a00c4
:101950000700350002003c000c08a3000400320020
:101960000601be0003f0a0000cf0a70019fd07005f
:101970000a85680001f0a1000af0a70001f0a000ac
:1019800085fe37000800be0083fe370010022000ed
:101990000cf0a6007042880083fe3700881f780094
:1019a000030478000300e00007003d006000100021
:1019b000e080180060011900e081190002003b007e
:1019c00001f02d000300370033fe070008f0a700e8
:1019d00001f0a0004f04780000000600020ab900e0
:1019e000001bb9000200b8008100420081004300e2
:1019f000000006006022b800060220000000d000af
:101a00008180d2000482d2008582d2000000a00032
:101a10000202520083825a00030031000202420097
:101a200083824a000000a1000603e900f3ff3a00a8
:101a30000000060031e2a90097c0a90097e0a900c4
:101a400087c0a90087e0a90000000600811180007e
:101a5000e6806000e68f50000c003a00030037007b
:101a60003322ab00feff3a00a1118800b0007800dd
:101a70000100e000faff3a00000006003322ab004c
:101a8000feff3a008100fb00a1118800b040780001
:101a90000104e000f9ff3a000000060000102000f9
:101aa0003202b6000000e9004f00de000000060030
:101ab00021e2a9009560a9009580a9008560a90090
:101ac0008580a9000000060001118000e68060000a
:101ad000e68f500001003200f00fb20020118800a4
:101ae000000006000c00fa00889fbe000004780089
:101af000f0ff2700d0bf9f008004eb0099bf9f003c
:101b000088bf9f00a8bf9f00200c2000b0bf9f008f
:101b100078815700cfb09700708057002a000700e7
:101b20000fb89700094878008fb8970008805000d8
:101b30004f04be000080fa00000006008000eb00a9
:101b400080f2880091f2880011c0b300e0e4210027
:101b50000148780000000600e0e421001004e000e5
:101b600002003a0010002000f4ff0700d2e6240033
:101b7000631c240080f2800091f2800097ff070030
:101b800092032300030020000001410081814900ed
:101b900082f2880093f288000300780000f0a10030
:101ba00000000600d0019000028151004240a900cf
:101bb0000300340010017800014978000208e800b1
:101bc0000100780000000600f6874700889fbe00ed
:101bd0008a9fbe008c9fbe008e1f78000005780093
:101be000a1b79f00020778008004eb008e02370047
:101bf000afb097008100e800a1b79f0051c2b300c9
:101c0000814f500003003a00afb097000004eb0092
:101c100011003700ba0090000000fb000168a3002b
:101c20000700320009017800800078000a0078007f
:101c3000dcff07000000e00005003a007a023700f0
:101c40008a00780084020700e10f4000760232002b
:101c50008904e800740237000100780031417800ff
:101c6000d3c2b300834f51000c00320007003c0088
:101c7000edc15100834f51000a003200ebc1410019
:101c8000834f51000d003a000800370003c3b30032
:101c9000834f510009003a00060037000830a000c9
:101ca000edff37000800a000ebff37000810a00090
:101cb000e9ff37000820a000e7ff37000810a70061
:101cc0000800a1000830a7000820a1008200fb0046
:101cd0000103b100e98f50000c003e0000017800c4
:101ce0008000eb006a08b900b201fb000303b100f9
:101cf00080804100020078009201fb000303b100e4
:101d0000e98f5100f7ff3600060037008000eb0036
:101d1000a3c2b300834f510002003a00ce00780006
:101d20000000e8008005eb00e2c2b300904f110014
:101d300009003a0008e0a00064415100d04f1100b2
:101d4000030032000001780001027800060037002d
:101d5000ce0578000000e800000178000900370097
:101d60006a58b9008085410002007800b201fb008a
:101d70000303b100e98f5100f9ff360084007800b9
:101d8000f5ff370032407800a2b79f00c3c6b3000a
:101d9000834f5000250032000f003c0032c6b300d4
:101da000824f50008800320004003c000004e00034
:101db000220232006b4151000f00370042c6b300cf
:101dc000824f50001700320065414100824f5000a1
:101dd00094003a001300370032c7b300824f50001e
:101de0001b00320007003c0064415100824f50004c
:101df000100032000241e800824f500089003a0092
:101e00000f00370052c7b300824f50008a003200e3
:101e100063414100824f500082003a00e0df9f00a2
:101e200009003700e0df9f00850037000840a00070
:101e3000d4ff3700e0df9f000860a000800037007b
:101e4000e0df9f000850a0000870a0007c00370071
:101e5000e0df9f004e007800000678000000e00000
:101e600001003a00ecd721000c0178000000eb00e3
:101e7000010037000000e800e24178000304e000c0
:101e8000fcff3a00800678000b00e00003003200ff
:101e90008d8f5500010031008b0678008005eb0026
:101ea0008d8f5000010036008d855000680464005d
:101eb0002a003a00110037003a0090000068a300a1
:101ec0000700320009017800010220000a007800b2
:101ed00034ff07000000e00006003a00060037006b
:101ee0008a00780000022000db010700e10f4000bb
:101ef000010032008904e8008b05e9000b00e000d6
:101f0000edff3a008085eb00140037003a009000a6
:101f10000068a300090032000c007800b000fb004c
:101f200000067800090178000a0078001dff07000c
:101f30000000e00008003a00080037008c0078003c
:101f40003100fb00010678008a007800c20107001a
:101f5000e10f4000010032008904e8000d00780024
:101f60008006e9000000e000e8ff3a000800e00019
:101f7000ad013200110037003a0090000068a30064
:101f80000700320009017800010220000a007800f1
:101f900004ff07000000e00006003a0006003700da
:101fa0008a00780000022000ab010700e10f40002a
:101fb000010032008904e8008b05e9000b00e00015
:101fc000edff3a00980137004e017800cf91de0016
:101fd000c81ade004818dd004812de000402700056
:101fe000e4df9f000848a300080032000404e0007a
:101ff00006003200e14f420004003200f4df9f008f
:1020000082e79f002d00200002003700f2df9f00d2
:102010001d002000e2fd2f000f0141000206e80034
:1020200099ff3700e0df9f00ecfd2f000f06460010
:102030001d00200094ff3700e0df9f00080cb30074
:1020400008017800020cb200700064000200e00099
:102050000d003a000000e000020032004e06be0013
:10206000020037004e067800cfe6de00e00f560093
:10207000e08f5e000a003d003800b30060061600e5
:10208000e0861e00060037000000e000020032007b
:102090004e06be00020037004e0678008006eb00b8
:1020a0000b00e00005003a008c8576000bf0a700dd
:1020b0008b05ea008b05e900cf5dde008801780022
:1020c000030cb200e3b79f0000042000808f510092
:1020d0002300320003003c000300e000080032004f
:1020e0002d003700000820006fb29700800f5200cb
:1020f0000d003200000c2000800f520026003a0034
:1021000062d8210010c0b30064014100b20f560034
:10211000a28f5e001f0039000040e800ea4f500027
:10212000f9ff3a001b00370010c0b3000201200085
:1021300003002000820f5600838f5e0015003900d7
:10214000441add00cc11de00830172004411dd0071
:102150000040e800e84f5000f6ff3a000d0037005d
:1021600010c0b3008200200003002000820f560040
:10217000838f5e0007003900431add00cd11de00b9
:10218000830172004311dd000040e800eb4f500076
:10219000f6ff3a00e0df9f006fd997000200fb00d6
:1021a0008b0f500002003d00ebdf9f000300370063
:1021b000808f550001003d00800578000100e0009f
:1021c0000300320063006400010032008100e90076
:1021d00008e8a300050032008b8f50000200340095
:1021e0008b805000010037008000eb00efd9970092
:1021f0000300fb000002eb00d4b79f00808f50006b
:102200000200340000805000d0b79f000828a300cf
:1022100040003200610164000818a3000f00320082
:102220003a0090000068a30006003200b1022000ce
:102230000200e000010032008180e800090178001e
:102240000d003700b00220000200e0000100320063
:102250000080e8008a0078000e0037000200e000ed
:10226000100032003a0090000068a300070032001e
:1022700009017800010220000a00780049fe0700e9
:102280000000e00006003a00060037008a007800ef
:1022900000022000f0000700e10f400001003200c2
:1022a0008904e8005fb097000000e0005a003200a7
:1022b000bcb79f00cdb79f00800678003a00900021
:1022c0000068a30007003200090178000103200024
:1022d0000a00780033fe07000000e00006003a0024
:1022e000060037008a00780000032000da000700ab
:1022f000e10f4000010032008904e8008d06e9008a
:10230000eeff3a00ddb79f003fb69700cfb69700cb
:1023100041003700dfb197000300e0001a003200ef
:102320000838a30018003a00bcb79f00cdb79f0043
:10233000830678003a0090000068a300070032008e
:1023400009017800010220000a00780015fe07004c
:102350000000e00006003a00060037008a0078001e
:1023600000022000bc000700e10f40000100320025
:102370008904e8008d06e900eeff3a00ddb79f0012
:102380003fb69700cfb69700610164000818a3001c
:102390000f0032003a0090000068a30006003200ef
:1023a000b10220000200e000010032008180e8005c
:1023b000090178000d003700b00220000200e000a3
:1023c000010032000080e8008a0078000e0037002b
:1023d0000200e000100032003a0090000068a30004
:1023e0000700320009017800010220000a0078008d
:1023f000ecfd07000000e00006003a000600370090
:102400008a0078000002200093000700e10f4000de
:10241000010032008904e8000b03e9006330b900d1
:1024200000017800b2b79f004233dd0060d8210080
:10243000000343008e01780093b79f0008077800df
:10244000060478005c0037008b05e90000042000da
:102450006fb29700800f52003800320003003c003a
:102460000400e000080032003e00370000082000b1
:10247000efb09700808f500020003200000c200049
:10248000808f500037003a000e48a3001000320041
:102490001802be000401be000c00be00f4b79f008d
:1024a00085bf9f0053fd0700e0df9f000000fb0099
:1024b000cf80de007fb297008fba97000401be0084
:1024c00046fd07000006560081865e0007003700c3
:1024d00018017800110009000286d800a20020002f
:1024e000110009000280d800e1df9f006fd997003a
:1024f0000243b000e2df9f001a003700d0d621006f
:102500000e58a30001003200c0d5210061d821007f
:10251000810054000c01be008100e900030033007b
:102520008301d1000281d300fbff3700ef0061007f
:10253000e0c07800e1df9f000a0037000c00be0019
:10254000bfb197008301e900030033008100d1008f
:102550000080d300fbff3700674060000043b000fd
:10256000e0df9f00ba0090006fda97000400fb00e4
:102570000168a3000700320009017800800078009c
:102580000a00780087fd07000000e00005003a001f
:10259000050037008a0078002f000700e10f400097
:1025a000010032008904e8003fb09700630050004a
:1025b000b0b79f00640454000b00e000a2ff3a0093
:1025c0000e0478001fb797000838a30016003200e9
:1025d000dfb097000100e000130034000104780030
:1025e0003a0090000068a30007003200090178005b
:1025f000010220000a0078006afd07000000e000e8
:1026000006003a00060037008a0078000002200029
:1026100011000700e10f4000010032008904e800ca
:102620000804e900eeff3a002fb19700124078004d
:10263000e0df9f000004e0006dfd3a000900780033
:102640004f0778004f06be004f05be004f04be0086
:102650006f01b10000000600889fbe0001047800f1
:10266000b80090008084eb000118a3003a0032000b
:10267000180190000198a30002003a000200e00057
:1026800035003a000190a0003104980080047800e1
:10269000f90fb2000200e00002003a0028009000aa
:1026a000000c7800ea8f540005003a000178a3007e
:1026b00003003a0088007800d0002000e6ff070001
:1026c00018009000d8009000810f50000b003200dd
:1026d0000000e8001004980018007800094878000d
:1026e000000ce80011c0b30040e52100014878006b
:1026f000ea8f540018003a0005003700880078007f
:1027000009407800170007008004780012003700a5
:10271000380090000088a3000f00320018019000dc
:10272000a80090004800900031f907009800900040
:10273000810f500004003200380090000003b30005
:10274000300498008084eb000000eb001004980037
:1027500028009000000c7800090078004f04be00ab
:10276000000006000200fa00889fbe00a0ff9f0044
:1027700001047800380090000068a30033003a009c
:10278000e200600005003a000003b3003004980046
:10279000110498000080eb002e003700d804900050
:1027a0000900e00006003a0012002000e680570011
:1027b000480090000ef90700190498002300370024
:1027c000a80090000100e00008003a0071e5210037
:1027d00021049800010c7800210020005104980089
:1027e000110498000030a0003004980018019000f7
:1027f000a800900048009000fdf807002800900015
:102800008080eb0011049800aff897000148780031
:10281000000ce8002ff89700ea4f50000b003a0038
:10282000380090000088a3000800320018019000d2
:10283000a800900048009000edf807000000eb00b1
:1028400010049800a8009000010c7800aff89700e1
:102850000100fb004f04be000080fa0000000600eb
:020000040000fa
:102860005265000063650000697600006564000041
:102870003a200000257800000a0d00000044000006
:10288000617400006151000075650000756500000d
:102890003a20000025580000202500007520000087
:1028a0002575000020250000752000002558000037
:1028b0000a0d000000000000452d000050550000ea
:1028c000434b000020520000414e000047450000ed
:1028d000204100004e44000020420000454100001d
:1028e000524900004e4700002053000054410000b0
:1028f00052540000454400000a0d00000000000092
:08290000257500002000000015
:020000040000fa
:10290800889fbe008a1f7800800478004801200054
:102918000a0220000800780031090700801c7800ae
:102928000804e8008a0f5400faff3a004f057800bf
:102938004f04be0000000600e05e2100f0ff070023
:10294800c05e2100f8014000d00078004209de0096
:1029580002885000830f5000fbff3a000000060079
:10296800889fbe00800478000104fb0074004400c6
:102978001b09070008044400e15e2100e1007c0017
:10298800010050004240a90002003400800c780089
:1029980001003700800ceb004f04be000000060069
:1029a800e202a800e222a800e802a800e822a800a3
:1029b800e982a800e9a2a800e9c2a800e9e2a80003
:1029c800c4a2a800c482a800c422a800c402a80007
:1029d800000006000000fb00cf80de00eb0f500077
:1029e800e08f580060003e00006001000b003700d7
:1029f80011003700170037001d003700230037008b
:102a0800290037002f003700350037003b0037001a
:102a180041003700470037004d003700e202a800a8
:102a280040062000000000000000e900fdff3a0019
:102a3800e202a9004c003700e222a800400620006c
:102a4800000000000000e900fdff3a00e222a900b2
:102a580045003700e802a8004006200000000000fa
:102a68000000e900fdff3a00e802a9003e00370037
:102a7800e822a80040062000000000000000e9004d
:102a8800fdff3a00e822a90037003700e982a800d4
:102a980040062000000000000000e900fdff3a00a9
:102aa800e982a90030003700e9a2a800400620000a
:102ab800000000000000e900fdff3a00e9a2a900bb
:102ac80029003700e9c2a8004006200000000000e5
:102ad8000000e900fdff3a00e9c2a9002200370022
:102ae800e9e2a80040062000000000000000e9001c
:102af800fdff3a00e9e2a9001b003700c4a2a800c4
:102b080040062000000000000000e900fdff3a0038
:102b1800c4a2a90014003700c482a80040062000ff
:102b2800000000000000e900fdff3a00c482a9008f
:102b38000d003700c422a800400620000000000055
:102b48000000e900fdff3a00c422a9000600370092
:102b5800c402a80040062000000000000000e900b0
:102b6800fdff3a00c402a90000000600889fbe00cd
:102b78008a9fbe008c9fbe008e1f78000004eb0069
:102b88000840780093ff07000804e800ec0f5400a1
:102b9800fbff3a007c08070013e1a9001221a900f5
:102ba80012c1a90080ff2f00a800b6000000a000f5
:102bb800400588008500a9009500a800f0fc2f00ba
:102bc8001221b6000a21ef00cfc2ab000400320088
:102bd80000fa2000700888000468ef00040037003d
:102be800506621007008880010c0b30004e8b700e0
:102bf80013e1a8000085200002040700403e2100e0
:102c08003e0407002b4821006a5621000004eb000f
:102c180088047800cc4921004d4b2100ce4c21007e
:102c2800094078006bff07000000eb00802d78005a
:102c380000367c0080367c0000377c00615421001f
:102c480080307c00400e200000c8b900429320006c
:102c580000004100eb03070010c0b300004d7800ee
:102c68008904e8000884e8006a054500ec8f5400f0
:102c7800ebff3a000c28ef001828ef000e28ef00b1
:102c88001028ef0012a8ef001428ef001628ef0014
:102c98001a28ef000628ef0027ff0700c85e21006a
:102ca800780544000b48290049512100d81f7800b5
:102cb8008b1f78000900780088fb0700090078005e
:102cc8007d050700e48757008a0f5400f7ff3a0094
:102cd800a1c0b30040512100014878000000e8007d
:102ce800d1c0b300014878000000e8000048eb00bc
:102cf80009007800700507004f0778004f06be00ee
:102d08004f05be004f04be0000000600e202a90005
:102d1800e222a900e802a900e822a900e982a900a4
:102d2800e9a2a900e9c2a900e9e2a900c4a2a90090
:102d3800c482a900c422a900c402a9000000060098
:102d48000000fb00cf80de00eb0f5000e08f580042
:102d580024003e00006001000b0037000c00370023
:102d68000d0037000e0037000f0037001000370045
:102d78001100370012003700130037001400370025
:102d88001500370016003700e202a90015003700c9
:102d9800e222a90013003700e802a9001100370059
:102da800e822a9000f003700e982a9000d003700ca
:102db800e9a2a9000b003700e9c2a9000900370001
:102dc800e9e2a90007003700c4a2a90005003700fe
:102dd800c482a90003003700c422a90001003700fb
:102de800c402a900000006000000fb00cf80de003e
:102df800eb0f5000e08f580024003e0000600100f7
:102e08000b0037000c0037000d0037000e003700ac
:102e18000f0037001000370011003700120037008c
:102e2800130037001400370015003700160037006c
:102e3800e202a80015003700e222a80013003700bc
:102e4800e802a80011003700e822a8000f003700a8
:102e5800e982a8000d003700e9a2a8000b0037009e
:102e6800e9c2a80009003700e9e2a8000700370016
:102e7800c4a2a80005003700c482a80003003700d8
:102e8800c422a80001003700c402a8000000060000
:102e98008000780000852000750307000000060008
:102ea80080007800008520005c0307000000060011
:102eb8008f02b000889fbe008a9fbe008c9fbe0014
:102ec8008e1f7800a0802000f1ff07000004e000ba
:102ed800d70132001a28ef0060408000e10f50004f
:102ee80030003200e20f5000750032000000e000b0
:102ef800c1003a005a40800045408000c64080002a
:102f080060562100c2492100430020008000eb00e8
:102f180001067800695421008045eb00010478001f
:102f28004e4b21000d01200017c0b30090cf1300b5
:102f380015003a008352de00e1826200e9837800de
:102f4800878f520005003a001202e8000409780051
:102f5800e60f5200050032000b0037000b487800de
:102f68000603e80008097800070037000809780018
:102f78000db77800c44c210008b27800c74f210073
:102f880088b378001c0020006a0040000281e80035
:102f98008180e8008301e800f88f5000e2ff3a00e2
:102fa800920037005a40800046408000ce408000a2
:102fb80060562100424b2100c349210044002000f3
:102fc8008000eb001c002000010478004b48210021
:102fd800cd4c21008e047800c9b79f001ec0b300f5
:102fe800904f17002a003a000453de006103630083
:102ff800830278001300e00004003a001700200064
:103008008709780086b578001900370088097800a4
:10301800eb837800870f5300100032009204780089
:10302800708714008e34dd00d9b79f006d87780053
:103038000e8744008eb67800920478000909e900ea
:103048000700e0000a003a00ce4f2100ee83780026
:103058008703e80007b77800050037008043eb00d6
:1030680007487800cfb497008904e800c9b79f00e3
:103078001200e00006003a004e0020000e09780019
:10308800880a7800454e210088b278002c0020007c
:103098006a0040000281e8008180e8008381e8003e
:1030a8000402e800f88f5000ccff3a004fb79700b1
:1030b80046408800ce4088006c4088004e003700ab
:1030c8005c40800047408000c6408000f6b79f0003
:1030d800e8408000d8b79f0060562100424b21008d
:1030e800c3492100444e2100450020008000eb0028
:1030f800c1b79f00cd4f21001a0020004e48210083
:103108000003780019c0b30090cf140027003a00dc
:103118008563de00e1836300030478001300e000a8
:1031280003003a008a09780007b778000f003700d3
:103138008004eb0089097800ee847800898f5300b9
:10314800050032009204e900893ddd00148a45003b
:1031580009097800050037008044eb000948780029
:10316800ffb497008904e800f9b79f00820478004b
:103178001200e0000d003a00ed85780094854500c6
:10318800ef85650005003a004abb9f00c64c210048
:1031980066837800d6b79f00cab79f000003eb008c
:1031a800060c780008012000880c78006a004000ae
:1031b8000281e8008180e8008381e8000482e80059
:1031c8008502e800f88f5000cdff3a00474088009c
:1031d800ffb49700c94088005fb79700ee408800a9
:1031e8004fb09700d0408800030037004540880062
:1031f800c64088006c408800c0408000ec0f50003a
:1032080012003a001a28ef001828ef00695621002a
:103218000004eb004a0e20004c93200010c0b300bd
:10322800804c78000c28ef000ac0b9000000460066
:10323800c1fc2f008f8040008d0207000804e800c1
:10324800ea844400ec0f5400f4ff3a00d0408000b8
:10325800e10f5000f6003a000004eb000608e20017
:10326800de003a00e1552100f1b79f00e2bb2100e2
:10327800c2b79f00e3be2100b3b79f00c4c0b3002c
:10328800c4e79f00080778008042eb00c5df9f0075
:103298000443780086e79f00feaf9f009eb79f001b
:1032a8006066b8000c05be000004eb00e8a79f00ac
:1032b800400e200000f4b90041932000088440002b
:1032c800080078007e0207000000e000fcff3a00da
:1032d800420e200002f0b900439320000080410014
:1032e800c1fc2f008f804000610207006fa2970089
:1032f800d4b79f000400e0002d0032001600200023
:10330800ffb29700950f130031003a006120b80012
:1033180077f607000004be00cfb397001701be0080
:1033280075f607000001be000a00be00a7f60700f8
:103338000005be003fb097001001be000800be00a7
:103348006df607000001be000c00be009ff60700e6
:103358000006be009fb097005fb19700828f5000b3
:1033680009003100cee79f000fe29700c4df9f00fd
:103378008ee79f0001037800f6af9f008203780074
:1033880097b79f00120037007fac9700dfb4970013
:10339800890f54000c003100cedf9f008fe09700aa
:1033a800c1e79f0009017800f2af9f0008003700cd
:1033b80014002000ffb19700930f120004003a0098
:1033c800cee79f00020037000fe39700c6e79f0093
:1033d8000e07e800ffb39700ea834300f7b79f00a2
:1033e8004fb4970064044400c8b79f00bfb4970067
:1033f800e4844400b9b79f00ec0f5700aaff3a00d5
:103408006011b8000a00be00cdf607006044b8009d
:103418000000e000040032000a01be000c00be00fb
:10342800c9f607000004be001fb797006170b80016
:103438002ff607000001be002ff607000001be00ae
:103448002df607000006be007fa997006110b8009e
:1034580027f607000001be0027f607000001be009e
:1034680025f60700d0b79f00e1b79f008fe29700cd
:103478000500fb004200dd00eec12100000047000e
:103488001001be000800be004ff60700cbf607008b
:103498000005be004fdb97000600fb004200dd0080
:1034a800000747001e01be000800be0046f60700e0
:1034b800c2f60700f0b79f0081bf9f000a01be0057
:1034c8000a00be000cf607000001be000c00be009a
:1034d800bcf607000005be007fb197008fb99700c2
:1034e8000200be0004f607000001be005fb09700ae
:1034f800efb09700b3f607000001be000a00be0057
:1035080032f60700f1f60700f0f607000005be00e6
:10351800e3408000f3a79f0002002400c361240059
:103528000800be00f4f507001df70700d0af9f00a4
:103538000448e20004003a000a00be0039f7070018
:10354800a0af9f00040037000a00be0035f707004f
:103558004200de00a0af9f001fb29700b4af9f00eb
:10356800cfe2970085df9f0088af9f0099af9f004b
:10357800ffa097000fa997009fa997002faa97006f
:103588009fb297004fab9700dfab9700403e2100fa
:10359800e0010700f50307000004e0000100320025
:1035a800740307001a28ef001828ef00605621005e
:1035b800830720008081410012c0b3008000eb0027
:1035c8000248780041b89f006a004000830f50000d
:1035d800fbff3a000c28ef00150037004a93200043
:1035e800e9552100400e200000c0b9000000450048
:1035f800b30107000000e000faff3a006a40b90092
:10360800e400400089804000420e200002c1b90059
:1036180002004500960107000804e800ec0f54007a
:10362800f0ff3a00e1408000e0552100a2040700c5
:103638004f0778004f06be004f05be004f04be007e
:103648008f02b1000000060080007800403e210093
:10365800d1010700000006000e00fa0090bf9f008d
:10366800a1bf9f00b2bf9f00c3bf9f00d4bf9f00f0
:10367800e5bf9f00f6bf9f00ee805700403e210047
:10368800c50107000080fa000000060006c8bf0058
:10369800000006000000fb00304088000000060023
:1036a80007e2a8000742a90070002000ac20b7007c
:1036b8008600a9009600a8000004290030108800a0
:1036c8000002200050108800550407000000060082
:1036d800881f78000000fb00cf80de00e202200097
:1036e800820f5000e08f580093003e0000600100f8
:1036f8002e00370030003700320037003300370023
:1037080035003700360037003800370039003700f9
:103718003b0037003c003700870037008600370041
:1037280085003700840037008300370082003700a7
:1037380081003700800037007f0037007e003700a7
:103748003400370037003700390037003a003700b7
:103758003c0037003d0037003f003700400037008d
:103768004200370043003700450037004600370065
:1037780048003700490037004b0037004c0037003d
:103788004e0037004f003700510037005200370015
:1037980054003700550037005700370058003700ed
:1037a8005a0037005b0037005d003700e0d4210085
:1037b800a5ff07006100370070ea80004800de00be
:1037c8005e00370070ea80005c003700d0ea8000b5
:1037d8004800de0059003700d0ea80005700370063
:1037e800a0ea80004800de0054003700a0ea80000c
:1037f80052003700b0ea80004800de004f00370072
:10380800b0ea80004d00370080d5210010407800d4
:103818004a003700c183200060cd21004e04070014
:1038280046003700d0e680004800de00430037003d
:10383800d0e680004100370020e780004800de0025
:103848003e00370020e780003c00370070e780002a
:103858004800de003900370070e780003700370085
:10386800c0e780004800de0034003700c0e7800071
:103878003200370010e880004800de002f003700d3
:1038880010e880002d00370060e880004800de0066
:103898002a00370060e8800028003700b0e8800080
:1038a8004800de0025003700b0e88000230037001c
:1038b80000e980004800de002000370000e98000b1
:1038c8001e00370050e980004800de001b0037006a
:1038d80050e9800019003700a0e980004800de00a8
:1038e80016003700a0e9800014003700f0e98000d6
:1038f8004800de0011003700f0e980000f003700b3
:1039080040ea80004800de000c00370040ea8000f2
:103918000a003700e04180004800de000700370059
:10392800f80f2000e0418000000464002e04070026
:1039380008407800010037000040eb004f04780091
:1039480000000600ef4f50004800320006003c001f
:10395800ed4f50003c0032003e003c00ec4f500060
:103968004c003a0006003700f14f50004300320087
:1039780040003500f24f500046003a004200370040
:10398800c084200001487800e0c6b30080cf500012
:1039980002003e004d68ef0047003700ffcf4000af
:1039a80026003e000181fb008001eb0026db2f0092
:1039b800f7ff2f000203530083835b000180fb00a5
:1039c8004300dd00cf80de00060240008782480009
:1039d8000211b8004a1bdd004610de00000073002b
:1039e800c698de000000520081805a00f04188002d
:1039f80001428800e00f5000e08f580003003d00ae
:103a08003e28ef004028ef0007003700320c200066
:103a1800820f5000e08f580003003400360c20005d
:103a2800f64188004028ef00e183200091407800ab
:103a3800d2842000014978001f00370030ccb30041
:103a48004de8b7001c003700014078003ae8b7009d
:103a5800190037008180fb003ac8bf004800dd002c
:103a680000804000eb010700130037001f0107002a
:103a780011003700b0fb07000f0037000140780045
:103a880004ff07000c003700014078004b020700d4
:103a980009003700eb4f500007003c008180fb0015
:103aa800a2832000124178004811dd008280400086
:103ab8000000fb000601070000000600c2442000c9
:103ac800020140008000eb0001097800930020000b
:103ad800e2442000033079000281e800020040003f
:103ae80001087800000006000003be00024520001f
:103af800e60279000001eb00e98f520017003c0054
:103b0800e3442000830143001302e800a2002000e0
:103b1800110009000202d80001017800820978002a
:103b280087007800430620000391b9000281e9006c
:103b3800820143000001eb0024032000b129780032
:103b48000201e800840f5100fcff3a000145200003
:103b5800010043000508e800120020000200780078
:103b680000000600881f7800000478000245200045
:103b7800e80179000001eb000300e00016003400c2
:103b8800c544200085024400240320001503780062
:103b980004b3b9008601410083814100e8987900a7
:103ba8000201e800840f5100f8ff3a00c1442000e8
:103bb800010244009401e800a2002000110009005d
:103bc8008201d800010a7800014520000100440064
:103bd8001008e90012002000020078004f04780065
:103be80000000600000178001000200001452000b8
:103bf800e28078000100e000010034000000eb00e2
:103c0800000006008000eb0071a89800d206200092
:103c180002b0980011b098000000060080027800f9
:103c28000103780095b190000001eb00d406200054
:103c3800848f51000c003c0005b190000201e8009f
:103c48000402e800110009000401d800010178000d
:103c580082b2980002014100863279008301e800af
:103c680093b29800120020000200780000000600bd
:103c78000002780094b190000001eb000300e0001e
:103c88000d00340074a9900002014100e408790095
:103c9800f4a890008100e800e20620001100090065
:103ca8008200d80071aa980094b090008100e900c1
:103cb80011b29800120020000200780000000600ef
:103cc800800078001000200091b090000100e00012
:103cd800010034000000eb000000060010b0900066
:103ce800000006008000eb0071a89800d2062000b2
:103cf80002b0980011b09800000006008000eb00a8
:103d08005188980092002000628898007188980075
:103d1800000006000e00fa00881f780000047800f2
:103d280081bf9f0092bf9f00a3bf9f00b4bf9f00a9
:103d3800c5bf9f00d6bf9f00e7bf9f00788990004e
:103d48008000eb00e90f51000f003c00e88890006c
:103d58008100e800a3002000110009008300d800ba
:103d6800618c98006e0ab900840044007080570086
:103d780006000900b0187800e100b1000201e8006f
:103d8800728c980011002000010078004f04780020
:103d98000080fa000000060000027800f489900014
:103da8000001eb000300e00010003400548990008b
:103db8006e11b9000200420006000900b018780030
:103dc800e100b100d48890008100e800a200200042
:103dd800110009008200d800518a9800f4889000e8
:103de8008100e900718a9800120020000200780022
:103df800000006008000780010002000f188900084
:103e08000100e000010034000000eb0000000600a3
:103e18008000eb00011898001118980021189800ec
:103e280000000600a01a90000001eb000500e00069
:103e38000a003c0012189800800178003182fb00cb
:103e4800841978000201e800ec0f5100fbff3a00ea
:103e58008502e8002518980012002000020078006a
:103e680000000600a01990000001eb000300e0002c
:103e78000e003400001a90006c22b9008401410041
:103e880083814100e0d879000201e800ec0f51007d
:103e9800f8ff3a008000eb0001189800a018900085
:103ea8008100e90021189800120020000200780023
:103eb800000006008000780010002000a118900083
:103ec8000100e000010034000000eb0000000600e3
:103ed8000000400002de21000131780012002000bd
:103ee80081df21008230780000000600ef0eb0006c
:103ef800889fbe008a9fbe008c9fbe008e1f7800e0
:103f08004cf02f000f0646006ef32f000f074700f6
:103f180020f32f000080470080bf9f000e0178002b
:103f28000c0078008000eb00012878000129780057
:103f38008fb99700830f5000fbff3a00e4fc2f0075
:103f48000f0242000483e9007c81570006007800d4
:103f58008000eb0001287800820f5000fdff3a0036
:103f680069df2100f9b79f0061e3210078814400ef
:103f7800090078008001eb001500200014002000e3
:103f8800d00f120003003a0011027800042add0065
:103f9800848141008180e800820f5000f7ff3a00d9
:103fa800b3079f00c31f9f00c3079f00d31f9f0035
:103fb800d3079f00e31f9f00adf02f008f864600b8
:103fc800ebf32f008f8545000005eb00dcb79f0061
:103fd800060678008e047800c9b79f0015003700e0
:103fe800540078000a00de00610060005801780083
:103ff8008204dd008981410019002000d58f14005a
:1040080004003a00800478000900a2000249dd009b
:104018009b0d4100d62b40008100e900f0ff3a00db
:10402800030f78000a05e8008b85e800f00f5500bb
:104038000c0032008d86e8000d0778009d0178009d
:10404800e0dd2100e0b79f0048e321008c03780001
:104058000c037800ffb2970000027800c10020002e
:10406800dfff37005fb697004fb79700ef13970051
:104078007f1397008f1a97001f1a9700ff2e97003b
:104088008f3097009f319700c3b79f00af349700d8
:10409800d9b79f000000eb00e8fc2f000f04440094
:1040a8006be321008adf2100bcb79f00010678007e
:1040b800e8007800ef806000f0801000013478009c
:1040c8006b017800c309de00e18161008219dd001f
:1040d80083834300c209de00e18161008219dd00ab
:1040e800030343008101d100e18161008219dd00f1
:1040f80083824200e1816000821cdd0009024200e7
:10410800ea047800e18f540014003a008180ea0044
:10411800c30cde00e1846400824cdd008986460021
:10412800c20cde00e1846400824cdd000906460012
:104138008100d100e18060008208dd00cfb49700e3
:1041480081844400c9b79f000300a2000219dd0062
:10415800dfb0970082804000d1b79f000080e80060
:10416800f80f5000d2ff3a008c0078003fb6970055
:10417800e7179f00f6179f00851f9f00941f9f0059
:10418800fd2f9f0081379f00cfb1970093379f0085
:104198005fb29700a4379f000000eb00a01f9f00ac
:1041a800b01f9f00b0379f00c0379f00a0f62f00b8
:1041b8000f0040005c087800de04780019009800c1
:1041c800640040008fb89700810f5600f9ff3a004d
:1041d800a0f62f000f004000e702070061df210072
:1041e8000000eb006fb19700ffb19700002978003d
:1041f80080297800810f5100fcff3a004f077800b2
:104208004f06be004f05be004f04be00ef0eb100c2
:1042180000000600e1dd210062df21007882400015
:10422800130020008028780003297800848f50002c
:10423800fcff3a002dff07000000060031e2a8004d
:1042480031a2a8003182a900f0cf2f003022b60099
:1042580030e2a90030c2a90030a2a9003082a9002a
:104268003062a90090ff2f003022b6003002a9006a
:1042780033e2a90033a2a90033c2a9003362a9001e
:104288003342a8003322a900f0f32f003222b600ef
:1042980032a2a900a0022000c011880087e0a9006e
:1042a80087c0a90097e0a80097c0a80000000600f2
:1042b800def5070000000600e2f50700f5f5070047
:1042c8000004e000fdff3a000000060020ac2100d9
:1042d8004cfe070021e2a80021a2a8002182a90023
:1042e800f0cf2f002022b60020e2a90020c2a900aa
:1042f80020a2a9002082a9002062a90090ff2f0017
:104308002022b6002002a90023e2a90023a2a900c6
:1043180023c2a9002362a9002342a8002322a900de
:10432800f0f32f002222b60022a2a900a00220004a
:10433800401188008580a9008560a900f1ff280048
:1043480040058000808060000000260001007000a9
:10435800400588009580a8009560a8003868ef009f
:1043680020ac21005ffe070000000600cef5070024
:1043780000000600889fbe0048ab210019c0b300aa
:1043880005003700b841880080832000094878007c
:104398001880fb00caf5070008007800aafc07008f
:1043a8000004e000f7ff3a004f04be0000000600da
:1043b80020ac21004bfe0700000006002ce8b700e7
:1043c800000006003c00fa00881f78000000eb009f
:1043d800a0bf9f00b0bf9f0020ac21003ffe070098
:1043e800e40f50005e003400ec80570020ac210040
:1043f8001ffe0700afb897008180fb00a00a2000cd
:10440800808f500056003a00e880570020ac210009
:1044180017fe07004fb89700f24f500050003e00bb
:10442800e680570020ac210011fe0700e480570009
:1044380020ac21000efe0700ea80570020ac2100c6
:104448000bfe0700bfb897008180fb0050052000d5
:10445800808f500042003a00801f7800f80f20003b
:104468005fb89700881f60003fb89700881f6000fa
:104478001fb89700881f60006fb09700881f600002
:10448800f0432900801f780060fb2f000f004000d8
:1044980092f5070060fb2f000f00400086ff070021
:1044a8006fb0970008046000ec875700ef0f5400c6
:1044b8000c00320005003e00ec0f54000d003200e5
:1044c800ee0f54001c003a0011003700f10f5400a1
:1044d8000c00320005003900f20f540016003a00b3
:1044e8001200370081fe07001d00370012f907008f
:1044f8001b0037005fb897000080fb0048020700e8
:10450800170037002ff8970062fc070014003700e7
:10451800efb897008180fb005fb897004800dd0086
:10452800008040003bff07000d0037002ff8970080
:10453800a2ff07000a003700eb0f540008003e00f6
:10454800f20f2000efb9970082816100dfb8970071
:10455800c808dd0081804100020060005cfe0700a1
:104568004f0478000080fa00000006002cc8bf0045
:044578000000060039
:020000040000fa
:10457c00d61c000086000000000000004c08000063
:10458c000200000002000000966c00003a080000d7
:10459c000c00000000000000361e00001800000097
:1045ac0002000000030004000005000008000900e0
:1045bc00000a00000b000c00000d00000e000f00a4
:1045cc0000000000e01d00003000000000000000b2
:1045dc00a61b0000a8000000020000000f00320023
:1045ec00004b000069008500009f00005bff790014
:1045fc00ff97ff00b3ffce00fff1ff00ed46770001
:10460c003fc18d00243fed0083843e00ed83840088
:10461c00be6c97002ebf1900ff6ebf00ed467700f1
:10462c00bff7040035bfed008384be008e596600d1
:10463c003ec18d00243fed0046773f00ed838400a2
:10464c003e761b00443fed0046773f00ed46770079
:10465c003f043a003b3f03007cb73e00ed838400ef
:10466c00bef7040035bfed004677bf0050707900ef
:10467c00bf761b0044bfed008384be00850a860014
:10468c003ef966005f3f37008da73f008192ea003c
:10469c003ffc8f001440cc009a314000874e38000c
:1046ac00c0e2cb0016c0810092eabf000305ac004b
:1046bc00bff966005fbf85000a86be005008000087
:1046cc00b60d000000000000000800001e000000f5
:1046dc000000000006160000ae0400000000000000
:1046ec001e0800000e000000000000004e1c000020
:1046fc0088000000000000004608000006000000d2
:10470c0000000000b41a0000f200000000000000dd
:10471c002c0800000e00000000000000ae1d000080
:10472c0032000000000000004e08000002000000f3
:10473c00000000004e1e00000600000000000000fb
:10474c005c1d0000520000000200000030313200fd
:10475c003334350036373800394142004344450084
:10476c0046003000313233003435360037383900ea
:10477c00616263006465660000286e00756c6c00f5
:10478c002900000001000000000a00000000640085
:10479c0000000000e8030000001027000000a0004b
:1047ac008601000040420f00008096009800000037
:1047bc00e1f5050000ca9a003b000000101e000045
:1047cc002600000002000000551e000000551e00cf
:1047dc000900000000020000571e000000571e00d8
:1047ec000e020100000000000000000000000000ac
:1047fc000602020000000000101e0000541e000003
:10480c0006000000000000005a1e0000020000001c
:0c481c000200000001000000000000008d
:020000040000fa
:104828000000eb0070e28800a0e2880080e28800c7
:1048380090e2880080e68800a0e6880090e688007c
:1048480080c5210082072000000141008000eb00a4
:1048580001087800310098001100980021009800a4
:104868006a004000820f5000f9ff3a004a68ef00e2
:1048780000000600ec8747008e1f7800a0bf9f004d
:10488800b1bf9f00c2bf9f00d3bf9f006c87570076
:104898003e00be0070e2880081e288001e00be0073
:1048a80090e28800a1e28800b4e288004f0778000f
:1048b800cf00b10000000600889fbe008001eb0019
:1048c80086c521008507200003014000030243003c
:1048d8003204be00088abe004400b000321a7800d4
:1048e800321278001201780022029800ea81410011
:1048f800858f5100f4ff3a004142880010c0b30090
:104908004ae8b7004f04be00000006000600fa009f
:10491800d0bf9f00e1bf9f005fb89700efb8970036
:1049280080e6880091e68800a2e688000080fa0008
:104938000000060072e2800083e280000298be0058
:1049480092e28000a3e280000298be00b3e28000f9
:104958000308780000000600889fbe000041eb00b5
:10496800a384200093417800e1cf510012003a005f
:104978008001eb0086c52100850720000301430064
:10498800030240003204be00088abe004400b000a2
:10499800321a780032127800120178002202980048
:1049a800ea814100858f5100f4ff3a0049428000b6
:1049b8008908780012c0b300024078004f04be0096
:1049c8000000060082e6800093e680000288be00b0
:1049d800a3e680002300980000000600e0c4210040
:1049e8000008eb00000006004a68ef00000006001f
:1049f80000cd21000008eb000000060030428800ce
:104a0800000006003042800000000600cdc2a80069
:104a18006800a800c662a900c682a900c6a2a900ab
:104a2800c702a900c722a900c742a900c762a900f6
:104a3800c782a900c7a2a900c7c2a900c7e2a900e6
:104a4800c602a900ca62a900ca82a900caa2a9000e
:104a5800cb02a900cb22a900cb42a900cb62a900b6
:104a6800cb82a900cba2a900cbc2a900cbe2a900a6
:104a7800ca02a900d282a800d2a2a800d2c2a80065
:104a8800d2e2a800d302a800d322a800d342a800eb
:104a9800d362a800d382a800d3a2a800d3c2a800da
:104aa800d3e2a800de02a900de22a900e402a900e0
:104ab800e422a900e582a900e5a2a900e5c2a900af
:104ac800e5e2a900c0a2a900c082a900c022a900ed
:104ad800c002a900e202a900e222a900e802a90096
:104ae800e822a900e982a900e9a2a900e9c2a9006f
:104af800e9e2a900c4a2a900c482a900c422a900ad
:104b0800c402a900c062a900df82a900c462a9008a
:104b1800e382a800e442a800e462a80040a7a90034
:104b280000052000303a8800f0f32f004427b60033
:104b380000fe2f004427b600a10920003200200003
:104b4800800720003374200080497800814978006c
:104b580082497800710520001200200060042000be
:104b680023742000804978008149780082497800c0
:104b78000200270001002300133a800003006100af
:104b8800810f5000fcff3a00000006001800fa00f0
:104b9800889fbe008a9fbe00fa0020000b002000fc
:104ba8000004eb00491f200021003700000000002e
:104bb8000000e900fdff3a0000fe2f000f00400052
:104bc8004ff707002fb09700bfb0970080806800ac
:104bd8001fb097000fb19700020068008080400066
:104be8004fb097005fb197000000690080804000d7
:104bf8006fb097007fb19700000069008080400087
:104c08000fb897001fb99700000069008080400026
:104c18002fb897003fb99700000069000080400056
:104c28000004440061055500e0855d000200320083
:104c380009007800ddff370008007800bdf30700a1
:104c48004f05be004f04be000080fa0000000600b9
:104c58006eff070092fa0700780007009bfd070027
:104c680076fd0700e0da2100c1452900220009008d
:104c7800315878003002b1003102b1008efd0700d2
:104c880036000700b9f70700c0ff070040062000fc
:104c980063000700c462a900c5fd0700c9fd07003d
:104ca80083f80700fdff370011e1a9001021a900d2
:104cb80010c1a9000621ef00f0fc2f001021b6005a
:104cc80080ff2f008421b60091052000610888002c
:104cd800c1022000110c8800010c88008461a90021
:104ce8008401b6006000b300200c8800f1ff2800a2
:104cf8003005800080806000000025000100700001
:104d08003005880084e0a90094e0a90011e1a8001a
:104d18002066210069fb07000000060005e1a900e4
:104d28000421a90004c1a900f0ff2800a400b600ce
:104d380000e0a000200588008460a9009460a80015
:104d4800f0fc2f000421b6000021ef0000fa20003b
:104d58001008880005e1a80000000600d2ff07003f
:104d6800eeff0700000006008000780020662100a2
:104d78007cfb070000000600800078002066210008
:104d880059fb070000000600f000200050198800b9
:104d9800f3ff21002032200010886100f1cf2f009e
:104da8000232200012896000000e20002023b70084
:104db8002043a9002143a800223220001289610063
:104dc8002343a90025e3a900a0c0b30024e3b7004a
:104dd80095a0a90021e3a800000006000000060035
:104de8007f00600001fe2f00421980008280600071
:104df80081007000411988002023a800803e20000f
:104e0800000000000000e900fdff3a002023a9008f
:104e18002003ab00feff32000018800000000600ef
:104e2800c842a90041128000401288004002ab002d
:104e3800feff3200c842a80000000600dee2a8001b
:104e4800df02a900c642a9006022ef004382a90040
:104e58004362a9004342a9004322a9004302a800d3
:104e680042e2a90042c2a90042a2a80030fe2f00d7
:104e78004222b600c0ff2f004202b6000000a00088
:104e88001012880000002800001288000000eb00c3
:084e9800e3ff07000000060023
:020000040000fa
:0200000401f009
:04000c00a000000050
:020000040000fa
:0200000401f009
:0400100045000000a7
:020000040000fa
:0200000401f009
:040014005f00000089
:00000001FF
